:020000040800F2
:1000000000060020E1010008E3010008E301000808
:10001000E3010008E3010008E3010008E301000830
:10002000E3010008E3010008E3010008A52F000830
:10003000E3010008E3010008E3010008E301000810
:10004000E3010008E3010008E3010008E301000800
:10005000E3010008E30100084D3200087532000892
:100060009D320008C5320008ED320008E3010008A7
:10007000E3010008E3010008E3010008E3010008D0
:10008000E3010008E3010008E3010008E3010008C0
:10009000E3010008E3010008E3010008153300084C
:1000A000E3010008E3010008E3010008E3010008A0
:1000B000E9330008E3010008E3010008E301000858
:1000C000E3010008E3010008E3010008E301000880
:1000D000E3010008E3010008E3010008E301000870
:1000E00079330008E3010008E3010008E301000898
:1000F000E3010008E3010008E3010008E301000850
:10010000E3010008E3010008E3010008E30100083F
:10011000E3010008E3010008E3010008E30100082F
:10012000E3010008E3010008E3010008E30100081F
:10013000E3010008E3010008E3010008E30100080F
:10014000E3010008E3010008E30100085927000863
:10015000E3010008E3010008E3010008E3010008EF
:10016000E3010008E3010008E3010008E3010008DF
:10017000E3010008E3010008E3010008E3010008CF
:10018000E3010008E3010008E3010008E3010008BF
:10019000E3010008E3010008E3010008E3010008AF
:1001A000E3010008E3010008E3010008E30100089F
:1001B000E3010008E3010008E3010008E30100088F
:1001C000E3010008E3010008E3010008E30100087F
:1001D000E3010008E3010008E3010008E30100086F
:1001E00002E000F000F8FEE772B6374880F30888B6
:1001F000364880F3098836483649086040F20000E6
:10020000CCF200004EF63471CEF200010860BFF36C
:100210004F8FBFF36F8F40F20000C0F2F0004EF638
:100220008851CEF200010860BFF34F8FBFF36F8F8C
:100230004FF00000E1EE100A4EF63C71CEF20001E4
:100240000860062080F31488BFF36F8F01F04CFF25
:1002500002F046FE4FF055301F491B4A91423CBF09
:1002600041F8040BFAE71D49184A91423CBF41F896
:10027000040BFAE71A491B4A1B4B9A423EBF51F83E
:10028000040B42F8040BF8E700201849184A914281
:100290003CBF41F8040BFAE701F02AFF02F074FEBC
:1002A000144C154DAC4203DA54F8041B8847F9E7A7
:1002B00000F042F8114C124DAC4203DA54F8041B22
:1002C0008847F9E701F012BF000600200022002055
:1002D0000000000808ED00E00000002000060020FB
:1002E000B0370008002200204022002040220020D9
:1002F000602E0020E0010008E0010008E001000895
:10030000E00100082DE9F04F2DED108AC1F80CD066
:10031000C3689D46BDEC108ABDE8F08F002383F3CF
:1003200011882846A047002001F08EFAFEE701F070
:100330001DFA00DFFEE7000038B500F06DFB01F0AC
:10034000A3FE054601F0C6FE0446D8B90F4B9D42F8
:100350001AD001339D4218BF044641F2883504BFCC
:1003600001240025002001F099FE0CB100F076F880
:1003700000F01CFD00F0B6FB284600F0C3F800F0CA
:100380006DF8F9E70025EDE70546EBE7010007B05A
:1003900008B500F079FBA0F120035842584108BD90
:1003A00007B541F21203022101A8ADF8043000F0B4
:1003B00089FB03B05DF804FB38B5302383F3118863
:1003C000174803680BB101F00BFB164A14480023D1
:1003D0004FF47A7101F0FAFA002383F31188124C7A
:1003E000236813B12368013B2360636813B163681A
:1003F000013B63600D4D2B7833B963687BB90220F4
:1004000000F046FC322363602B78032B07D163682E
:100410002BB9022000F03CFC4FF47A73636038BDC6
:1004200040220020B9030008602300205822002049
:10043000084B187003280CD8DFE800F00805020804
:10044000022000F015BC022000F002BC024B00228A
:100450005A6070475822002060230020244B254A10
:1004600010B51C461968013140D004339342F9D1CC
:100470006268214B9A4239D9204B9B6803F1006393
:1004800003F580339A4231D2002000F045FB022070
:10049000FFF7CEFF1A4B1A6C00221A64196E1A6607
:1004A000196E596C5A64596E5A665A6E5A6942F0FE
:1004B00080025A615A6922F080025A615A691A69A7
:1004C00042F000521A611A6922F000521A611B6947
:1004D00072B64FF0E0233021C3F8084DD4E9003262
:1004E00081F311889D4683F30888104710BD00BF33
:1004F0000000010820000108FFFF00080022002082
:10050000003802402DE9F04F93B0AA4B0090202212
:10051000FF210AA89D6800F0F3FBA74A1378A3B94E
:10052000A648012103601170302383F3118803680A
:100530000BB101F055FAA24AA04800234FF47A719A
:1005400001F044FA002383F31188009B13B19D4B03
:10055000009A1A609C4A009C1378032B1EBF00234C
:100560001370984A4FF0000A18BF5360D34656469E
:10057000D146012000F07CFB24B1924B1B68002B7C
:1005800000F01182002000F07FFA0390039B002B03
:10059000F2DB012000F05CFB039B213B162BE8D82B
:1005A00001A252F823F000BF050600082D0600083E
:1005B000C1060008730500087305000873050008EC
:1005C0004B0700081B0900083508000897080008B9
:1005D000BF080008E508000873050008F7080008D0
:1005E0007305000869090008A506000873050008DE
:1005F000AD09000811060008A506000873050008EB
:10060000970800080220FFF7C3FE002840F0F5819C
:10061000009B0221BAF1000F08BF1C4605A841F259
:100620001233ADF8143000F04DFAA2E74FF47A70AF
:1006300000F02AFA071EEBDB0220FFF7A9FE0028D4
:10064000E6D0013F052F00F2DA81DFE807F0030A68
:100650000D10133605230593042105A800F032FA86
:1006600017E054480421F9E758480421F6E75848B0
:100670000421F3E74FF01C08404600F04FFA08F160
:1006800004080590042105A800F01CFAB8F12C0F0D
:10069000F2D1012000FA07F747EA0B0B5FFA8BFB58
:1006A0004FF0000900F078FB26B10BF00B030B2B89
:1006B00008BF0024FFF774FE5BE746480421CDE73E
:1006C000002EA5D00BF00B030B2BA1D10220FFF7BE
:1006D0005FFE074600289BD0012000F01DFA022093
:1006E000FFF7A6FE00261FFA86F8404600F024FA1F
:1006F000044690B10021404600F02EFA0136002851
:10070000F1D1BA46044641F21213022105A8ADF810
:1007100014303E4600F0D6F92BE70120FFF788FEA3
:100720002546244B9B68AB4207D9284600F0F6F9D2
:10073000013040F067810435F3E7234B00251D703D
:10074000204BBA465D603E46ACE7002E3FF460AFFA
:100750000BF00B030B2B7FF45BAF0220FFF768FE5F
:10076000322000F091F9B0F10008FFF651AF18F017
:1007700003077FF44DAF0F4A926808EB05039342DD
:100780003FF646AFB8F5807F3FF742AF124B01937B
:10079000B84523DD4FF47A7000F076F90390039AA0
:1007A000002AFFF635AF019B039A03F8012B0137AE
:1007B000EDE700BF002200205C2300204022002043
:1007C000B9030008602300205822002004220020E2
:1007D000082200200C2200205C220020C820FFF705
:1007E000D7FD074600283FF413AF1F2D11D8C5F1E0
:1007F000200242450AAB25F0030028BF4246834948
:100800000192184400F056FA019A8048FF2100F046
:1008100077FA4FEAA8037D490193C8F38702284677
:1008200000F076FA064600283FF46DAF019B05EB19
:10083000830537E70220FFF7ABFD00283FF4E8AE61
:1008400000F0B6F900283FF4E3AE0027B846704B3D
:100850009B68BB4218D91F2F11D80A9B01330ED0B9
:1008600027F0030312AA134453F8203C0593404693
:10087000042205A900F0C4FA04378046E7E73846A9
:1008800000F04CF90590F2E7CDF81480042105A89A
:1008900000F018F906E70023642104A8049300F08F
:1008A00007F900287FF4B4AE0220FFF771FD00289D
:1008B0003FF4AEAE049800F063F90590E6E700233C
:1008C000642104A8049300F0F3F800287FF4A0AE9C
:1008D0000220FFF75DFD00283FF49AAE049800F077
:1008E0005FF9EAE70220FFF753FD00283FF490AEDE
:1008F00000F06EF9E1E70220FFF74AFD00283FF41F
:1009000087AE05A9142000F069F904210746049078
:1009100004A800F0D7F83946B9E7322000F0B4F85F
:10092000071EFFF675AEBB077FF472AE384A9268B9
:1009300007EB090393423FF66BAE0220FFF728FD59
:1009400000283FF465AE27F003074F44B9453FF454
:10095000A9AE484600F0E2F80421059005A800F091
:10096000B1F809F10409F1E74FF47A70FFF710FDCF
:1009700000283FF44DAE00F01BF9002844D00A9B3C
:1009800001330BD008220AA9002000F0C1F9002889
:100990003AD02022FF210AA800F0B2F9FFF700FDAB
:1009A0001C4800F057FF13B0BDE8F08F002E3FF455
:1009B0002FAE0BF00B030B2B7FF42AAE0023642128
:1009C00005A8059300F074F8074600287FF420AED0
:1009D0000220FFF7DDFC804600283FF419AEFFF748
:1009E000DFFC41F2883000F035FF059800F006FA90
:1009F000464600F0D1F93C46BBE5064652E64FF0CC
:100A0000000905E6BA467EE637467CE65C22002011
:100A100000220020A08601007047000070B50F4B37
:100A20001B780133DBB2012B0C4611D80C4D296821
:100A30004FF47A730E6AA2FB03320146224628461F
:100A4000B047844204D1074B00221A70012070BDC8
:100A50004FF4FA7000F0FEFE0020F8E710220020AC
:100A6000082600209423002070B504464FF47A76BF
:100A7000412C254628BF412506FB05F000F0EAFE83
:100A8000641BF5D170BD000007B5002302460121AB
:100A90000DF107008DF80730FFF7C0FF20B19DF87A
:100AA000070003B05DF804FB4FF0FF30F9E70000EA
:100AB0000A4608B50421FFF7B1FF80F00100C0B27B
:100AC000404208BD30B4054C2368DD69044B0A463A
:100AD000AC460146204630BC604700BF08260020D7
:100AE000A086010070B501F0D5F9094E094D30809E
:100AF000002428683388834208D901F0C5F92B689F
:100B000004440133B4F5803F2B60F2D370BD00BFC5
:100B1000962300206823002001F06ABA00F10060EB
:100B200000F580300068704700F10060920000F529
:100B3000803001F0F5B90000054B1A68054B1B88A1
:100B40009B1A834202D9104401F09EB900207047DD
:100B5000682300209623002038B5084D044629B1AB
:100B600028682044BDE8384001F0AEB92868204428
:100B700001F092F90028F3D038BD00BF68230020AF
:100B800010F003030AD1B0F5047F05D200F1005044
:100B9000A0F51040D0F80038184670470023FBE756
:100BA00000F10050A0F51040D0F8100A7047000086
:100BB000064991F8243033B10023086A81F82430C3
:100BC0000822FFF7B1BF0120704700BF6C2300204F
:100BD000014B1868704700BF002004E070B5194B46
:100BE0001D68194B0138C5F30B0408442D0C042271
:100BF0001E88A6420BD15C680A46013C824213461D
:100C00000FD214F9016F4EB102F8016BF6E7013A09
:100C100003F10803ECD181420B4602D22C2203F8E7
:100C2000012B0A4A05241688AE4204D1984284BF9B
:100C3000967803F8016B013C02F10402F3D1581AD3
:100C400070BD00BF002004E0CC340008B8340008B8
:100C5000022804D1054B4FF080429A617047012869
:100C6000FCD1024B4FF00052F7E700BF00000240FA
:100C7000022804D1054B4FF480429A617047012845
:100C8000FCD1024B4FF40052F7E700BF00000240D6
:100C9000022805D1064A536983F4804353617047A3
:100CA0000128FCD1024A536983F40053F6E700BFE0
:100CB0000000024010B50023934203D0CC5CC45422
:100CC0000133F9E710BD000010B5013810F9013FFC
:100CD0003BB191F900409C4203D11AB10131013A74
:100CE000F4E71AB191F90020981A10BD1046FCE7FC
:100CF00003460246D01A12F9011B0029FAD17047A7
:100D000002440346934202D003F8011BFAE77047FE
:100D10002DE9F8431F4D144695F8242007468846D0
:100D200052BBDFF870909CB395F824302BB9202289
:100D3000FF2148462F62FFF7E3FF95F82400C0F13A
:100D40000802A24228BF2246D6B24146920005EBD5
:100D50008000FFF7AFFF95F82430A41B1E44F6B2C5
:100D6000082E17449044E4B285F82460DBD1FFF7E5
:100D70001FFF0028D7D108E02B6A03EB82038342D0
:100D8000CFD0FFF715FF0028CBD10020BDE8F883B6
:100D90000120FBE76C230020024B1A78024B1A70EB
:100DA000704700BF942300201022002010B5104C83
:100DB000104800F0B5F821460E4800F0DDF8246830
:100DC000626DD2F8043843F00203C2F804384FF4DD
:100DD0007A70FFF749FE0849204600F0D3F9626DAA
:100DE000D2F8043823F00203C2F8043810BD00BF63
:100DF0009835000808260020A0350008704700003C
:100E000030B5094D0A4491420DD011F8013B5840CC
:100E1000082340F30004013B2C4013F0FF0384EA55
:100E20005000F6D1EFE730BD2083B8ED026843688B
:100E30001143016003B118477047000013B5446BBC
:100E4000D4F894341A681178042915D1217C022928
:100E500012D11979128901238B4013420CD101A9B7
:100E600004F14C0001F0F8FED4F89444019B217980
:100E70000246206800F0D0F902B010BD143001F035
:100E80007BBE00004FF0FF33143001F075BE000050
:100E90004C3001F04DBF00004FF0FF334C3001F0FB
:100EA00047BF0000143001F049BE00004FF0FF3191
:100EB000143001F043BE00004C3001F019BF0000B7
:100EC0004FF0FF324C3001F013BF0000002070479C
:100ED00010B5D0F894341A6811780429044617D153
:100EE000017C022914D15979528901238B40134284
:100EF0000ED1143001F0DCFD024648B1D4F8944420
:100F00004FF4807361792068BDE8104000F072B939
:100F100010BD0000406BFFF7DBBF00007047000012
:100F20007FB5124B036000234360C0E90233012503
:100F300002260F4B057404460290019300F18402CF
:100F4000294600964FF48073143001F08DFD094B53
:100F50000294CDE9006304F523724FF480732946AF
:100F600004F14C0001F054FE04B070BDEC340008F4
:100F7000150F00083D0E00080B68302282F311881F
:100F80000A7903EB820290614A79093243F8220020
:100F90008A7912B103EB820398610223C0F894149A
:100FA0000374002080F311887047000038B5037F78
:100FB000044613B190F85430ABB9201D012502212D
:100FC000FFF734FF04F1140025776FF0010100F002
:100FD00069FC84F8545004F14C006FF00101BDE845
:100FE000384000F05FBC38BD10B501210446043024
:100FF000FFF71CFF0023237784F8543010BD000056
:1010000038B504460025143001F046FD04F14C00CB
:10101000257701F015FE201D84F854500121FFF7BB
:1010200005FF2046BDE83840FFF752BF90F8443036
:1010300003F06003202B07D190F84520212A4FF0C0
:10104000000303D81F2A06D800207047222AFBD1AC
:10105000C0E90E3303E0034A82630722C2630364DC
:10106000012070471122002037B5D0F894341A6857
:101070001178042904461AD1017C022917D1197963
:10108000128901238B40134211D100F14C052846EF
:1010900001F096FE58B101A9284601F0DDFDD4F813
:1010A0009444019B21790246206800F0B5F803B012
:1010B00030BD0000F0B500EB810385B09E690446A9
:1010C0000D46FEB1302383F3118804EB8507301DF4
:1010D0000821FFF7ABFEFB685B691B6806F14C005B
:1010E0001BB1019001F0C6FD019803A901F0B4FD08
:1010F000024648B1039B2946204600F08DF80023A4
:1011000083F3118805B0F0BDFB685A691268002AA4
:10111000F5D01B8A013B1340F1D104F14402EAE708
:10112000093138B550F82140DCB1302383F3118800
:10113000D4F894241368527903EB8203DB689B692B
:101140005D6845B104216018FFF770FE294604F17F
:10115000140001F0B7FC2046FFF7BAFE002383F32A
:10116000118838BD7047000001F016B801230370E4
:101170000023C0E90133C36183620362C362436237
:101180000363704738B50446302383F31188002584
:10119000C0E90355C0E90555416001F00DF802238F
:1011A000237085F31188284638BD000070B500EB28
:1011B000810305465069DA600E46144618B11022C4
:1011C0000021FFF79DFDA06918B110220021FFF753
:1011D00097FD31462846BDE8704001F0B7B80000E1
:1011E000826802F0011282600022C0E9042282615A
:1011F00001F038B9F0B400EB81044789E4680125B7
:10120000A4698D403D43458123600023A260636053
:10121000F0BC01F053B90000F0B400EB8104078981
:10122000E468012564698D403D4305812360002306
:10123000A2606360F0BC01F0CDB9000070B502237C
:10124000002504460370C0E90255C0E90455C56491
:10125000856180F8345001F015F863681B6823B18C
:1012600029462046BDE87040184770BD0378052B1D
:1012700010B504460AD080F8503005230370436847
:101280001B680BB1042198470023A36010BD000028
:101290000178052906D190F85020436802701B6838
:1012A00003B118477047000070B590F83430044619
:1012B00013B1002380F8343004F14402204601F0D9
:1012C000F3F863689B68B3B994F8443013F0600591
:1012D00035D00021204601F093FB0021204601F08B
:1012E00085FB63681B6813B10621204698470623D7
:1012F00084F8343070BD204698470028E4D0B4F814
:101300004A30E26B9A4288BFE36394F94430E56B5C
:10131000002B4FF0300380F20381002D00F0F280AB
:10132000092284F8342083F311880021D4E90E23A4
:101330002046FFF771FF002383F31188DAE794F862
:10134000452003F07F0343EA022340F20232934236
:1013500000F0C58021D8B3F5807F48D00DD8012B8F
:101360003FD0022B00F09380002BB2D104F14C024D
:10137000A2630222E2632364C1E7B3F5817F00F038
:101380009B80B3F5407FA4D194F84630012BA0D1C7
:10139000B4F84C3043F0020332E0B3F5006F4DD0A7
:1013A00017D8B3F5A06F31D0A3F5C063012B90D847
:1013B000636894F846205E6894F84710B4F84830A3
:1013C0002046B047002884D04368A3630368E363E2
:1013D0001AE0B3F5106F36D040F6024293427FF424
:1013E00078AF5C4BA3630223E3630023C3E794F865
:1013F0004630012B7FF46DAFB4F84C3023F002037C
:10140000C4E90E55A4F84C30256478E7B4F84430AC
:10141000B3F5A06F0ED194F8463084F84E302046D4
:1014200000F088FF63681B6813B1012120469847CC
:10143000032323700023C4E90E339CE704F14F0318
:10144000A3630123C3E72378042B10D1302383F354
:1014500011882046FFF7C4FE85F3118803216368D5
:1014600084F84F5021701B680BB12046984794F8C0
:101470004630002BDED084F84F300423237063689D
:101480001B68002BD6D0022120469847D2E794F85B
:1014900048301D0603F00F0120460AD500F0F6FF84
:1014A000012804D002287FF414AF2B4B9AE72B4B72
:1014B00098E700F0DDFFF3E794F84630002B7FF467
:1014C00008AF94F8483013F00F01B3D01A06204645
:1014D00002D501F0A9FAADE701F09CFAAAE794F869
:1014E0004630002B7FF4F5AE94F8483013F00F012E
:1014F000A0D01B06204602D501F082FA9AE701F03F
:1015000075FA97E7142284F8342083F311882B4668
:101510002A4629462046FFF76DFE85F31188E9E645
:101520005DB1152284F8342083F311880021D4E9B9
:101530000E232046FFF75EFEFDE60B2284F83420E2
:1015400083F311882B462A4629462046FFF764FE7E
:10155000E3E700BF1C350008143500081835000803
:1015600038B590F834300446002B3ED0063BDAB252
:101570000F2A34D80F2B32D8DFE803F03731310887
:10158000223231313131313131313737C56BB0F839
:101590004A309D4214D2C3681B8AB5FBF3F203FBA9
:1015A00012556DB9302383F311882B462A462946FC
:1015B000FFF732FE85F311880A2384F834300EE0F9
:1015C000142384F83430302383F3118800231A461F
:1015D00019462046FFF70EFE002383F3118838BD1D
:1015E000036C03B198470023E7E70021204601F090
:1015F00007FA0021204601F0F9F963681B6813B16E
:101600000621204698470623D7E7000010B590F83A
:101610003430142B044629D017D8062B05D001D816
:101620001BB110BD093B022BFBD80021204601F065
:10163000E7F90021204601F0D9F963681B6813B16E
:10164000062120469847062319E0152BE9D10B23E4
:1016500080F83430302383F3118800231A4619466A
:10166000FFF7DAFD002383F31188DAE7C3689B698B
:101670005B68002BD5D1036C03B19847002384F835
:101680003430CEE700230375826803691B689968CC
:101690009142FBD25A680360426010605860704704
:1016A00000230375826803691B6899689142FBD81F
:1016B0005A680360426010605860704708B5084679
:1016C000302383F311880B7D032B05D0042B0DD021
:1016D0002BB983F3118808BD8B6900221A604FF083
:1016E000FF338361FFF7CEFF0023F2E7D1E9003239
:1016F00013605A60F3E70000FFF7C4BF054BD968D9
:101700000875186802681A60536001220275D86073
:10171000FEF7F8BD9823002030B50C4BDD684B1C5C
:1017200087B004460FD02B46094A684600F04EF9B0
:101730002046FFF7E3FF009B13B1684600F050F925
:10174000A86907B030BDFFF7D9FFF9E7982300205B
:10175000BD160008044B1A68DB6890689B689842C5
:1017600094BF00200120704798230020084B10B53B
:101770001C68D86822681A60536001222275DC60F8
:10178000FFF78EFF01462046BDE81040FEF7BABDC8
:101790009823002038B5074C074908480123002545
:1017A0002370656001F044FB0223237085F31188E8
:1017B00038BD00BF002600202435000898230020F3
:1017C00000F044B9034A516853685B1A9842FBD849
:1017D000704700BF001000E08B60022308618B821D
:1017E000084670478368A3F1840243F8142C026909
:1017F00043F8442C426943F8402C094A43F8242C0E
:10180000C26843F8182C022203F80C2C002203F8BB
:101810000B2C044A43F8102CA3F12000704700BFA2
:101820001D0300089823002008B5FFF7DBFFBDE883
:101830000840FFF761BF0000024BDB6898610F2092
:10184000FFF75CBF98230020302383F31188FFF754
:10185000F3BF000008B50146302383F31188082048
:10186000FFF75AFF002383F3118808BD064BDB689E
:1018700039B1426818605A60136043600420FFF772
:101880004BBF4FF0FF307047982300200368984209
:1018900006D01A680260506099611846FFF72CBFA5
:1018A0007047000038B504460D462068844200D1D8
:1018B00038BD036823605C608561FFF71DFFF4E7B6
:1018C00010B503689C68A2420CD85C688A600B6003
:1018D0004C602160596099688A1A9A604FF0FF3312
:1018E000836010BD1B68121BECE700000A2938BF9B
:1018F0000A2170B504460D460A26601901F092FAD5
:1019000001F07EFA041BA54203D8751C2E4604463E
:10191000F3E70A2E04D9BDE87040012001F0C8BAEF
:1019200070BD0000F8B5144B0D46D96103F11001EC
:1019300041600A2A1969826038BF0A220160486042
:101940001861A818144601F05FFA0A2701F058FA46
:10195000431BA342064606D37C1C281901F062FAF9
:1019600027463546F2E70A2F04D9BDE8F8400120A2
:1019700001F09EBAF8BD00BF98230020F8B50646D6
:101980000D4601F03DFA0F4A134653F8107F9F426F
:1019900006D12A4601463046BDE8F840FFF7C2BFEF
:1019A000D169BB68441A2C1928BF2C46A34202D91E
:1019B0002946FFF79BFF224631460348BDE8F84021
:1019C000FFF77EBF98230020A823002010B4C0E9B1
:1019D000032300235DF8044B4361FFF7CFBF0000F2
:1019E00010B5194C236998420DD0D0E900328168B6
:1019F00013605A609A680A449A60002303604FF0AB
:101A0000FF33A36110BD2346026843F8102F5360D3
:101A10000022026022699A4203D1BDE8104001F021
:101A2000FBB9936881680B44936001F0E9F922697E
:101A3000E1699268441AA242E4D91144BDE8104019
:101A4000091AFFF753BF00BF982300202DE9F04784
:101A5000DFF8BC8008F110072C4ED8F8105001F0C8
:101A6000CFF9D8F81C40AA68031B9A423ED8144408
:101A7000D5E900324FF00009C8F81C4013605A60E5
:101A8000C5F80090D8F81030B34201D101F0C4F984
:101A900089F31188D5E9033128469847302383F329
:101AA00011886B69002BD8D001F0AAF96A69A0EB04
:101AB00004094A4582460DD2022001F0F9F90022BC
:101AC000D8F81030B34208D151462846BDE8F04757
:101AD000FFF728BF121A2244F2E712EB090938BFB8
:101AE0004A4629463846FFF7EBFEB5E7D8F81030EE
:101AF000B34208D01444211AC8F81C00A960BDE8FC
:101B0000F047FFF7F3BEBDE8F08700BFA823002031
:101B10009823002000207047FEE700007047000077
:101B20004FF0FF307047000002290CD0032904D089
:101B30000129074818BF00207047032A05D8054827
:101B400000EBC2007047044870470020704700BF98
:101B5000FC35000820220020B035000870B59AB08E
:101B60000546084601A9144600F0C2F801A8FFF78F
:101B7000BFF8431C5B00C5E9003400222370032337
:101B80006370C6B201AB02341046D1B28E4204F18A
:101B9000020401D81AB070BD13F8011B04F8021C2E
:101BA00004F8010C0132F0E708B5302383F3118803
:101BB0000348FFF759FA002383F3118808BD00BFDB
:101BC0000826002090F8443003F01F02012A07D1B4
:101BD00090F845200B2A03D10023C0E90E3315E00D
:101BE00003F06003202B08D1B0F848302BB990F8EF
:101BF0004520212A03D81F2A04D8FFF717BA222A22
:101C0000EBD0FAE7034A82630722C2630364012030
:101C1000704700BF1822002007B5052917D8DFE854
:101C200001F0191603191920302383F31188104A83
:101C300001900121FFF7BAFA01980E4A0221FFF73D
:101C4000B5FA0D48FFF7DCF9002383F3118803B0E0
:101C50005DF804FB302383F311880748FFF7A6F9EA
:101C6000F2E7302383F311880348FFF7BDF9EBE770
:101C700050350008743500080826002038B50C4D92
:101C80000C4C0D492A4604F10800FFF767FF05F1E7
:101C9000CA0204F110000949FFF760FF05F5CA7296
:101CA00004F118000649BDE83840FFF757BF00BFF0
:101CB000D02A002020220020303500083A350008C4
:101CC0004535000870B5044608460D46FFF710F884
:101CD000C6B22046013403780BB9184670BD3246AF
:101CE0002946FEF7F1FF0028F3D10120F6E70000B6
:101CF0002DE9F04705460C46FEF7FAFF2B49C6B220
:101D00002846FFF7DFFF08B10736F6B22849284614
:101D1000FFF7D8FF08B11036F6B2632E0BD8DFF804
:101D20008C80DFF88C90234FDFF894A02E7846B992
:101D30002670BDE8F08729462046BDE8F04701F04F
:101D40009DBB252E2ED1072241462846FEF7BCFF1B
:101D500070B9194B224603F10C0153F8040B42F8F9
:101D6000040B8B42F9D11B88138007350E34DDE755
:101D7000082249462846FEF7A7FF98B90F4BA21C38
:101D8000197809090232C95D02F8041C13F8011B15
:101D900001F00F015345C95D02F8031CF0D118345E
:101DA0000835C3E704F8016B0135BFE71C360008AE
:101DB000453500083336000824360008107AFF1F26
:101DC0001C7AFF1FBFF34F8F024AD368DB03FCD49A
:101DD000704700BF003C024008B5094B1B7873B93F
:101DE000FFF7F0FF074B1A69002ABFBF064A5A6087
:101DF00002F188325A601A6822F480621A6008BDC3
:101E00002E2D0020003C02402301674508B50B4BF6
:101E10001B7893B9FFF7D6FF094B1A6942F00042CD
:101E20001A611A6842F480521A601A6822F48052C9
:101E30001A601A6842F480621A6008BD2E2D0020D4
:101E4000003C02400B28F0B516D80C4C0C49237806
:101E50007BB90C4D0E460C234FF0006255F8047B05
:101E600046F8042B013B13F0FF033A44F6D101235B
:101E7000237051F82000F0BD0020FCE7602D002009
:101E8000302D002044360008014B53F820007047E5
:101E9000443600080C2070470B2810B5044601D9C1
:101EA000002010BDFFF7CEFF064B53F82430184436
:101EB000C21A0BB90120F4E712680132F0D1043BD9
:101EC000F6E700BF443600080B2810B5044621D8B9
:101ED000FFF778FFFFF780FF0F4AF323D360C300BB
:101EE000DBB243F4007343F002031361136943F45C
:101EF00080331361FFF766FFFFF7A4FF074B53F82A
:101F0000241000F0D9F8FFF781FF2046BDE810400B
:101F1000FFF7C2BF002010BD003C0240443600085D
:101F2000F8B512F00103144642D18218B2F1016FE4
:101F300057D82D4B1B6813F0010352D02B4DFFF7E0
:101F40004BFFF323EB60FFF73DFF40F20127032C2B
:101F500015D824F001046618244C401A40F20117E9
:101F6000B142236900EB010524D123F00103236171
:101F7000FFF74CFF0120F8BD043C0430E7E783077E
:101F8000E7D12B6923F440732B612B693B432B6111
:101F900051F8046B0660BFF34F8FFFF713FF036820
:101FA0009E42E9D02B6923F001032B61FFF72EFF3E
:101FB0000020E0E723F44073236123693B4323615E
:101FC0000B882B80BFF34F8FFFF7FCFE2D8831F875
:101FD000023BADB2AB42C3D0236923F001032361BE
:101FE000E4E71846C7E700BF00380240003C024063
:101FF000084908B50B7828B11BB9FFF7EDFE01239E
:102000000B7008BD002BFCD0BDE808400870FFF73E
:10201000FDBE00BF2E2D002010B50244064BD2B2EB
:10202000904200D110BD441C00B253F8200041F88A
:10203000040BE0B2F4E700BF502800400F4B30B56E
:102040001C6F240407D41C6F44F400741C671C6FBD
:1020500044F400441C670A4C236843F480732360F3
:102060000244084BD2B2904200D130BD441C00B2B1
:1020700051F8045B43F82050E0B2F4E70038024026
:10208000007000405028004007B5012201A900203F
:10209000FFF7C2FF019803B05DF804FB13B50446D7
:1020A000FFF7F2FFA04205D0012201A90020019410
:1020B000FFF7C4FF02B010BD70470000034B1A6861
:1020C0001AB9034AD2F874281A607047642D0020A8
:1020D0000030024008B5FFF7F1FF024B1868C0F36B
:1020E000407008BD642D002070470000FEE700002E
:1020F0000A4B0B480B4A90420BD30B4BDA1C121ABB
:10210000C11E22F003028B4238BF00220021FEF7DD
:10211000F7BD53F8041B40F8041BECE7F037000848
:10212000602E0020602E0020602E002070B5D0E9C7
:1021300015439E6800224FF0FF3504EB4213510116
:10214000D3F800090028BEBFD3F8000940F0804052
:10215000C3F80009D3F8000B0028BEBFD3F8000B6A
:1021600040F08040C3F8000B013263189642C3F878
:102170000859C3F8085BE0D24FF00113C4F81C38CB
:1021800070BD0000890141F02001016103699B06D7
:10219000FCD41220FFF716BB10B5054C2046FEF705
:1021A000E5FF4FF0A0436365024BA36510BD00BF80
:1021B000682D00209836000870B50378012B05467D
:1021C00050D12A4B446D98421BD1294B5A6B42F097
:1021D00080025A635A6D42F080025A655A6D5A69FC
:1021E00042F080025A615A6922F080025A610E213F
:1021F00043205B6900F022FC1E4BE3601E4BC4F8D9
:1022000000380023C4F8003EC02323606E6D4FF4F5
:102210000413A3633369002BFCDA012333610C2020
:10222000FFF7D0FA3369DB07FCD41220FFF7CAFAB4
:102230003369002BFCDA0026A6602846FFF776FFFC
:102240006B68C4F81068DB68C4F81468C4F81C68CC
:102250004BB90A4BA3614FF0FF336361A36843F0AE
:102260000103A36070BD064BF4E700BF682D00209A
:10227000003802404014004003002002003C30C0FF
:10228000083C30C0F8B5446D054600212046FFF7F4
:1022900079FFA96D00234FF001128F68C4F834381C
:1022A0004FF00066C4F81C284FF0FF3004EB4312D7
:1022B00001339F42C2F80069C2F8006BC2F80809F6
:1022C000C2F8080BF2D20B686A6DEB6563621023EB
:1022D0001361166916F01006FBD11220FFF772FA8F
:1022E000D4F8003823F4FE63C4F80038A36943F43B
:1022F000402343F01003A3610923C4F81038C4F845
:1023000014380A4BEB604FF0C043C4F8103B084B45
:10231000C4F8003BC4F81069C4F80039EB6D03F150
:10232000100243F48013EA65A362F8BD7436000816
:1023300040800010426D90F84E10D2F8003823F41F
:10234000FE6343EA0113C2F8003870472DE9F843F1
:1023500000EB8103456DDA68166806F00306731E0C
:10236000022B05EB41130C4680460FFA81F94FEA28
:1023700041104FF00001C3F8101B4FF0010104F1B0
:10238000100398BFB60401FA03F391698EBF334E70
:1023900006F1805606F5004600293AD0578A04F126
:1023A0005801490137436F50D5F81C180B43C5F845
:1023B0001C382B180021C3F8101953690127611E1E
:1023C000A7409BB3138A928B9B08012A88BF534373
:1023D000D8F85C20981842EA034301F1400205EB6B
:1023E0008202C8F85C00214653602846FFF7CAFE07
:1023F00008EB8900C3681B8A43EA845348346401AC
:102400001E432E51D5F81C381F43C5F81C78BDE873
:10241000F88305EB4917D7F8001B21F40041C7F8F2
:10242000001BD5F81C1821EA0303C0E704F13F03A1
:1024300005EB83030A4A5A6028462146FFF7A2FEAD
:1024400005EB4910D0F8003923F40043C0F80039F7
:10245000D5F81C3823EA0707D7E700BF0080001033
:1024600000040002826D1268C265FFF75FBE0000C3
:102470005831436D49015B5813F4004004D013F404
:10248000001F0CBF02200120704700004831436D3F
:1024900049015B5813F4004004D013F4001F0CBF33
:1024A000022001207047000000EB8101CB68196A0F
:1024B0000B6813604B6853607047000000EB8103AA
:1024C00030B5DD68AA691368D36019B9402B84BFA1
:1024D000402313606B8A1468426D1C44013CB4FBBA
:1024E000F3F46343033323F0030302EB411043EAA5
:1024F000C44343F0C043C0F8103B2B6803F0030310
:10250000012B09B20ED1D2F8083802EB411013F4B6
:10251000807FD0F8003B14BF43F0805343F000535A
:10252000C0F8003B02EB4112D2F8003B43F00443F9
:10253000C2F8003B30BD00002DE9F041244D6E6D26
:1025400006EB40130446D3F8087BC3F8087B380732
:102550000AD5D6F81438190706D505EB84032146A9
:10256000DB6828465B689847FA071FD5D6F8143809
:10257000DB071BD505EB8403D968CCB98B69488A86
:102580005A68B2FBF0F600FB16228AB91868DA68BE
:1025900090420DD2121AC3E90024302383F311882C
:1025A0000B482146FFF78AFF84F31188BDE8F081CC
:1025B000012303FA04F26B8923EA02036B81CB68DF
:1025C000002BF3D021460248BDE8F041184700BF78
:1025D000682D002000EB810370B5DD68436D6C69E8
:1025E0002668E6604A0156BB1A444FF40020C2F840
:1025F00010092A6802F00302012A0AB20ED1D3F8A8
:10260000080803EB421410F4807FD4F8000914BFCB
:1026100040F0805040F00050C4F8000903EB421233
:10262000D2F8000940F00440C2F80009D3F8340899
:10263000012202FA01F10143C3F8341870BD19B93F
:10264000402E84BF4020206020682E8A8419013CDF
:10265000B4FBF6F440EAC44040F000501A44C6E728
:102660002DE9F8433B4D6E6D06EB40130446D3F85D
:102670000889C3F8088918F0010F4FEA40171AD0EB
:10268000D6F81038DB0716D505EB8003D9684B69FF
:102690001868DA68904230D2121A4FF000091A60B6
:1026A000C3F80490302383F3118821462846FFF7AE
:1026B00091FF89F3118818F0800F1CD0D6F83438B8
:1026C0000126A640334216D005EB84036D6DD3F886
:1026D0000CC0DCF814200134E4B2D2F800E005EBC1
:1026E00004342F445168714515D3D5F8343823EAA2
:1026F0000606C5F83468BDE8F883012303FA04F23E
:102700002B8923EA02032B818B68002BD3D021462F
:1027100028469847CFE7BCF81000AEEB0103834290
:1027200028BF0346D7F8180980B2B3EB800FE2D870
:102730009068A0F1040959F8048FC4F80080A0EB58
:1027400009089844B8F1040FF5D818440B44906078
:102750005360C7E7682D00202DE9F74FA24C656D47
:102760006E69AB691E4016F480586E6107D0204632
:10277000FEF764FD03B0BDE8F04F00F047BC002E4B
:1027800012DAD5F8003E98489B071EBFD5F8003EE8
:1027900023F00303C5F8003ED5F8043823F0010305
:1027A000C5F80438FEF774FD370505D58E48FFF7E8
:1027B000BDFC8D48FEF75AFDB0040CD5D5F808389D
:1027C00013F0060FEB6823F470530CBF43F410535F
:1027D00043F4A053EB6031071BD56368DB681BB97A
:1027E000AB6923F00803AB612378052B0CD1D5F836
:1027F000003E7D489A071EBFD5F8003E23F0030334
:10280000C5F8003EFEF744FD6368DB680BB176480F
:102810009847F30274D4B70227D5D4F85490DFF860
:10282000C8B100274FF0010A09EB4712D2F8003B6C
:1028300003F44023B3F5802F11D1D2F8003B002BD5
:102840000DDA62890AFA07F322EA0303638104EBD3
:102850008703DB68DB6813B1394658469847A36D98
:1028600001379B68FFB29F42DED9F00617D5676D2E
:102870003A6AC2F30A1002F00F0302F4F012B2F542
:10288000802F00F08580B2F5402F08D104EB830340
:102890000022DB681B6A07F5805790426AD130033B
:1028A000D5F8184813D5E10302D50020FFF744FE00
:1028B000A20302D50120FFF73FFE630302D50220E9
:1028C000FFF73AFE270302D50320FFF735FE750315
:1028D0007FF550AFE00702D50020FFF7C1FEA1074A
:1028E00002D50120FFF7BCFE620702D50220FFF7E8
:1028F000B7FE23077FF53EAF0320FFF7B1FE39E7B0
:10290000636DDFF8E4A0019300274FF00109A36D88
:102910009B685FFA87FB9B453FF67DAF019B03EB0E
:102920004B13D3F8001901F44021B1F5802F1FD1CA
:10293000D3F8001900291BDAD3F8001941F09041AF
:10294000C3F80019D3F800190029FBDB5946606D64
:10295000FFF718FC218909FA0BF321EA030323810D
:1029600004EB8B03DB689B6813B1594650469847CC
:102970000137CCE7910708BFD7F80080072A98BF36
:1029800003F8018B02F1010298BF4FEA182884E78F
:10299000023304EB830207F580575268D2F818C05F
:1029A000DCF80820DCE9001CA1EB0C0C00218842BB
:1029B0000AD104EB830463689B699A6802449A60B5
:1029C0005A6802445A606AE711F0030F08BFD7F84B
:1029D00000808C4588BF02F8018B01F1010188BF9E
:1029E0004FEA1828E3E700BF682D0020436D03EB92
:1029F0004111D1F8003B43F40013C1F8003B70478C
:102A0000436D03EB4111D1F8003943F40013C1F8D1
:102A100000397047436D03EB4111D1F8003B23F4BB
:102A20000013C1F8003B7047436D03EB4111D1F82F
:102A3000003923F40013C1F80039704700F16043F6
:102A400003F561430901C9B283F80013012200F0C4
:102A50001F039A4043099B0003F1604303F5614360
:102A6000C3F880211A60704730B5039C01720433AB
:102A700004FB0325C0E90653049B03630021059B67
:102A8000C160C0E90000C0E90422C0E90842C0E911
:102A90000A11436330BD0000416A0022C0E90411FD
:102AA000C0E90A22C2606FF00101FEF7FBBE000020
:102AB000D0E90432934201D1C2680AB9181D7047A7
:102AC0000020704703691960C2680132C260C269A0
:102AD000134482690361934224BF436A0361002166
:102AE000FEF7D4BE38B504460D46E3683BB16269D3
:102AF000131D1268A3621344E362002007E0237AE7
:102B000033B929462046FEF7B1FE0028EDDA38BD7C
:102B10006FF00100FBE70000C368C269013BC360BE
:102B20004369134482694361934224BF436A43610A
:102B300000238362036B03B11847704770B53023DD
:102B4000044683F31188866A3EB9FFF7CBFF05463A
:102B500018B186F31188284670BDA36AE26A13F89B
:102B6000015BA362934202D32046FFF7D5FF002307
:102B700083F31188EFE700002DE9F84F04460E4675
:102B8000174698464FF0300989F311880025AA4668
:102B9000D4F828B0BBF1000F09D141462046FFF719
:102BA000A1FF20B18BF311882846BDE8F88FD4E946
:102BB0000A12A7EB050B521A934528BF9346BBF1A7
:102BC000400F1BD9334601F1400251F8040B43F882
:102BD000040B9142F9D1A36A40334036A3624035D9
:102BE000D4E90A239A4202D32046FFF795FF8AF3DD
:102BF0001188BD42D8D289F31188C9E730465A46B8
:102C0000FEF758F8A36A5B445E44A3625D44E7E7BD
:102C100010B5029C0172043303FB0421C0E90613C2
:102C20000023C0E90A33039B0363049BC460C0E92B
:102C30000000C0E90422C0E90842436310BD00005F
:102C4000026AC260426AC0E904220022C0E90A2284
:102C50006FF00101FEF726BED0E904239A4201D1AC
:102C6000C26822B9184650F8043B0B607047002335
:102C70001846FAE7C368C2690133C3604369134465
:102C800082694361934224BF436A43610021FEF796
:102C9000FDBD000038B504460D46E3683BB123692D
:102CA0001A1DA262E2691344E362002007E0237A5E
:102CB00033B929462046FEF7D9FD0028EDDA38BDA4
:102CC0006FF00100FBE7000003691960C268013A78
:102CD000C260C269134482690361934224BF436A9C
:102CE000036100238362036B03B118477047000040
:102CF00070B530230D460446114683F31188866A69
:102D00002EB9FFF7C7FF10B186F3118870BDA36A13
:102D10001D70A36AE26A01339342A36204D3E1699E
:102D200020460439FFF7D0FF002080F31188EDE73B
:102D30002DE9F84F04460D46904699464FF0300A6B
:102D40008AF311880026B346A76A4FB94946204640
:102D5000FFF7A0FF20B187F311883046BDE8F88F58
:102D6000D4E90A073A1AA8EB0607974228BF174684
:102D7000402F1BD905F1400355F8042B40F8042BD4
:102D80009D42F9D1A36A4033A3624036D4E90A23B5
:102D90009A4204D3E16920460439FFF795FF8BF38B
:102DA00011884645D9D28AF31188CDE729463A469B
:102DB000FDF780FFA36A3B443D44A3623E44E5E740
:102DC000D0E904239A4217D1C3689BB1836A8BB1BF
:102DD000043B9B1A0ED01360C368013BC360C369F8
:102DE0001A44836902619A4224BF436A0361002343
:102DF00083620123184670470023FBE700F030B9D7
:102E00004FF08043586A70474FF080430022586368
:102E10001A610222DA6070474FF080430022DA60C4
:102E2000704700004FF0804358637047FEE7000092
:102E300070B51B4B01630025044686B0586085625F
:102E40000E4600F0BFF804F11003C4E904334FF05C
:102E5000FF33C4E90635C4E90044A560E562FFF725
:102E6000CFFF2B460246C4E9082304F134010D4A82
:102E7000256580232046FEF7AFFC0123E0600A4A67
:102E80000375009272680192B268CDE90223074B84
:102E90006846CDE90435FEF7C7FC06B070BD00BF3B
:102EA00000260020A4360008A93600082D2E0008B0
:102EB000024AD36A1843D062704700BF98230020AB
:102EC0004B6843608B688360CB68C3600B69436168
:102ED0004B6903628B6943620B68036070470000B3
:102EE00008B5264B26481A6940F2FF110A431A61B9
:102EF0001A6922F4FF7222F001021A611A691A6B30
:102F00000A431A631A6D0A431A651E4A1B6D11465D
:102F1000FFF7D6FF02F11C0100F58060FFF7D0FF3C
:102F200002F1380100F58060FFF7CAFF02F1540199
:102F300000F58060FFF7C4FF02F1700100F58060CA
:102F4000FFF7BEFF02F18C0100F58060FFF7B8FFCC
:102F500002F1A80100F58060FFF7B2FF02F1C401A1
:102F600000F58060FFF7ACFF02F1E00100F5806042
:102F7000FFF7A6FFBDE8084000F0EEB800380240B9
:102F800000000240B036000808B500F059FAFEF71C
:102F900001FCFFF793F8BDE80840FEF76FBE0000A4
:102FA00070470000EFF3098305494A6B22F00102E4
:102FB0004A63683383F30988002383F311887047D9
:102FC00000EF00E0302080F3118862B60C4B0D4A10
:102FD000D96821F4E0610904090C0A43DA60D3F8E6
:102FE000FC20094942F08072C3F8FC200A6842F0D4
:102FF00001020A602022DA7783F82200704700BFBE
:1030000000ED00E00003FA05001000E010B53023E9
:1030100083F311880E4B5B6813F4006314D0F1EE58
:10302000103AEFF30984683C4FF08073E361094B79
:10303000DB6B236684F30988FEF78CFB10B1064B2B
:10304000A36110BD054BFBE783F31188F9E700BFCF
:1030500000ED00E000EF00E02F030008320300085D
:103060000F4B1A6C42F001021A641A6E42F0010210
:103070001A660C4A1B6E936843F0010393604FF08D
:10308000804353229A624FF0FF32DA6200229A6143
:103090005A63DA605A6001225A611A60704700BFB1
:1030A00000380240002004E04FF0804208B511696A
:1030B000D3680B40D9B2C9439B07116107D53023B0
:1030C00083F31188FEF77CFB002383F3118808BD8E
:1030D0001F4B1A696FEAC2526FEAD2521A611A691B
:1030E000C2F308021A614FF0FF301A695A69586139
:1030F00000215A6959615A691A6A62F080521A624B
:103100001A6A02F080521A621A6A5A6A58625A6A35
:1031100059625A6A1A6C42F080521A641A6E42F06E
:1031200080521A661A6E0B4A106840F48070106064
:10313000186F00F44070B0F5007F1EBF4FF4803070
:1031400018671967536823F40073536000F054B98B
:103150000038024000700040334B4FF080521A6438
:10316000324A4FF4404111601A6842F001021A607D
:103170001A689107FCD59A6822F003029A602A4BDC
:103180009A6812F00C02FBD1196801F0F90119607C
:103190009A601A6842F480321A601A689203FCD569
:1031A0005A6F42F001025A671F4B5A6F9007FCD5C5
:1031B0001F4A5A601A6842F080721A601B4A5368AC
:1031C0005904FCD5184B1A689201FCD5194A9A602B
:1031D000194B1A68194B9A42194B21D1194A116897
:1031E000194A91421CD140F205121A60144A136820
:1031F00003F00F03052BFAD10B4B9A6842F0020241
:103200009A609A6802F00C02082AFAD15A6C42F4C9
:1032100080425A645A6E42F480425A665B6E70472E
:1032200040F20572E1E700BF003802400070004044
:103230000854400700948838002004E011640020FE
:10324000003C024000ED00E041C20F41074A08B5D2
:10325000536903F00103536123B1054A13680BB1AD
:1032600050689847BDE80840FFF7D0BE003C0140D9
:10327000E02D0020074A08B5536903F002035361AB
:1032800023B1054A93680BB1D0689847BDE8084060
:10329000FFF7BCBE003C0140E02D0020074A08B506
:1032A000536903F00403536123B1054A13690BB159
:1032B00050699847BDE80840FFF7A8BE003C0140B0
:1032C000E02D0020074A08B5536903F00803536155
:1032D00023B1054A93690BB1D0699847BDE808400E
:1032E000FFF794BE003C0140E02D0020074A08B5DE
:1032F000536903F01003536123B1054A136A0BB1FC
:10330000506A9847BDE80840FFF780BE003C014086
:10331000E02D0020164B10B55C6904F478725A61F8
:10332000A30604D5134A936A0BB1D06A9847600686
:1033300004D5104A136B0BB1506B9847210604D586
:103340000C4A936B0BB1D06B9847E20504D5094A40
:10335000136C0BB1506C9847A30504D5054A936CC8
:103360000BB1D06C9847BDE81040FFF74FBE00BFCF
:10337000003C0140E02D0020194B10B55C6904F4BD
:103380007C425A61620504D5164A136D0BB1506D2B
:103390009847230504D5134A936D0BB1D06D984718
:1033A000E00404D50F4A136E0BB1506E9847A10488
:1033B00004D50C4A936E0BB1D06E9847620404D5C5
:1033C000084A136F0BB1506F9847230404D5054A80
:1033D000936F0BB1D06F9847BDE81040FFF716BE52
:1033E000003C0140E02D002008B5FFF75DFEBDE880
:1033F0000840FFF70BBE0000062108B50846FFF79E
:103400001DFB06210720FFF719FB06210820FFF707
:1034100015FB06210920FFF711FB06210A20FFF703
:103420000DFB06211720FFF709FB06212820FFF7D7
:1034300005FBBDE8084007211C20FFF7FFBA00008C
:1034400008B5FFF745FE00F00BF8FDF78DFEFDF720
:1034500065FDFFF7A5FDBDE80840FFF7CFBC000004
:103460000023054A19460133102BC2E9001102F16D
:103470000802F8D1704700BFE02D0020034611F884
:10348000012B03F8012B002AF9D1704753544D3317
:1034900032463F3F3F0053544D333246343078007C
:1034A00053544D3332463432780053544D33324600
:1034B0003434365858000000012033000010410019
:1034C00001105A00031059000710310000000000DD
:1034D0008C3400081304000096340008190400001E
:1034E000A034000821040000AA34000800000000F5
:1034F000990E0008850E0008C10E0008AD0E0008E8
:10350000B90E0008A50E0008910E00087D0E0008F7
:10351000CD0E0008000000000100000000000000C7
:103520006330000020350008F02300200026002032
:103530004172647550696C6F740025424F4152446A
:10354000252D424C002553455249414C2500000091
:103550000200000000000000B51000082111000862
:1035600040004000A02A0020B02A002002000000F5
:1035700000000000030000000000000065110008CA
:103580000000000010000000C02A00200000000021
:103590000100000000000000682D00200101020071
:1035A000191C0008291B0008C51B0008A91B0008DE
:1035B00043000000B835000809024300020100C0C2
:1035C0003209040000010202010005240010010577
:1035D00024010001042402020524060001070582DB
:1035E000030800FF09040100020A000000070501AA
:1035F00002400000070581024000000012000000A8
:10360000043600081201100102000040091241575F
:1036100000020102030100000403090425424F4196
:103620005244250041746F6D5243463430354E414B
:103630005649003031323334353637383941424318
:1036400044454600004000000040000000400000EB
:103650000040000000000100000002000000020025
:103660000000020000000200000002000000020052
:103670000000020000000000A91200086115000807
:103680000D16000840004000C82D0020C82D002065
:1036900001000000D82D0020800000004001000043
:1036A000030000006D61696E0069646C65000000D4
:1036B0000001801600000000AAAAAAAA00010000CA
:1036C000FF9F00000000000000A00A0000100001A1
:1036D00000000000AAAAAAAA00100001FFFF000033
:1036E00000000000000000000000000000000000DA
:1036F000AAAAAAAA00000000FFFF00000000000024
:10370000000000000000000000000000AAAAAAAA11
:1037100000000000FFFF00000000000000000000AB
:103720000000000000000000AAAAAAAA00000000F1
:10373000FFFF00000000000000000000000000008B
:1037400000000000AAAAAAAA00000000FFFF0000D3
:103750000000000000000000000000000000000069
:10376000AAAAAAAA00000000FFFF000000000000B3
:103770000000000000000000000000000A0000003F
:103780000000000003000000000000000000000036
:103790000000000000000000000000000000000029
:1037A0000000000000000000000000000000000019
:1037B000360400000000000000000F0000000000C0
:1037C000FF009600000000080096000000000800BE
:1037D000040000001836000800000000000000008F
:1037E00000000000000000000000000000000000D9
:00000001FF
